:020000040800F2
:10100000003C0020C140000809410008894E00084A
:101010008D4E0008914E0008954E0008000000001B
:10102000000000000000000000000000994E0008D1
:101030009D4E000800000000A14E0008A54E0008CB
:101040000941000809410008094100080941000858
:10105000094100080941000809410008255000081D
:1010600000000000A94E000809410008D14E000808
:10107000814F0008094100080941000800000000F4
:10108000015000080941000800000000C94F000895
:10109000E94F0008D94F000809410008094100083C
:1010A000094100080941000809410008FD4F0008F6
:1010B00009410008000000000000000000000000DE
:0C10C00009410008000000000941000880
:1010CC0053B94AB9002908BF00281CBF4FF0FF31A3
:1010DC004FF0FF3000F00CB8ADF1080C6DE904CE08
:1010EC0004F06AFEDDF804E0DDE9022304B0704789
:1010FC00704700BF10B5054C237833B9044B13B1BE
:10110C000448AFF300800123237010BD3808002081
:10111C0000000000EC60000808B5034B1BB103494C
:10112C000348AFF3008008BD000000003C0800201D
:10113C00EC600008AF4BB04AB3F87CC018882DE9BE
:10114C00F04FACEB00011588AC4C89B24A098D42CA
:10115C0087B02180628080F0E580A94D2D888D427A
:10116C0040F2E0805968DFF89C820F1AD3E9020143
:10117C00BFB2081A80B2BA422CBF002701278242A4
:10118C002CBF002101210591A160D3E90451A1EBF1
:10119C00050ED3E90651A1EB050AD3E908511FFA54
:1011AC008EFE1FFA8AFA7245A1EB050189B22CBF9B
:1011BC004FF0000E4FF0010E52452CBF4FF0000ABD
:1011CC004FF0010A8A422CBF002101210491616178
:1011DC00D3E90A51491B89B28A42D3E90C51A1EBDC
:1011EC00050189B22CBF002001208A422CBF0025AA
:1011FC0001250295E561D3E90E51491B89B28A425A
:10120C00D3E91051A1EB050189B22CBF00260126B0
:10121C008A422CBF4FF0000B4FF0010B0390A061E2
:10122C00019626626760C4F80CE0C4F810A0C4F8FC
:10123C0024B0D3E912514D1BD3E914618E1B00214C
:10124C00A8F80010D3E91A01ADB2B6B2AA42A1EBCC
:10125C00000189B22CBF00250125B2422CBF00260B
:10126C0001268A422CBF002101214FEA8108A1638B
:10127C00D3E91691A1EB0909D3E918011FFA89F9F1
:10128C00091A89B24A452CBF4FF000094FF00109E9
:10129C008A422CBF0021012148EAC1086163996F81
:1012AC000398C4F83090ACEB010189B28A422CBF90
:1012BC000021012148EA01082164D3E91C31CB1A31
:1012CC009BB29A422CBF00230123E36348EA4308F4
:1012DC00059B4D49A56243406B409A00049B0198C5
:1012EC00E6627B408BEA030342EAC30380EA0A020C
:1012FC0089EA0209029A43EA090382EA0E0986EA9C
:10130C00090943EA49090B787BB1404B1B7883B937
:10131C00C84513D0B4F8543000220133A4F854302B
:10132C0084F8482007B0BDE8F08F384B1A78002AB3
:10133C0076D0C8F10F085FFA88F8E9E7B4F84630C0
:10134C0030480133A4F84630236B0022012B028075
:10135C0004BF2F4A1370059B049A5B0243EA872350
:10136C00334343EA0E2343EACA1343EA8213039A34
:10137C0043EA4213029A43EA0213019A43EAC20374
:10138C0094F8482043EA8B0343EA4505FAB92F2D1C
:10139C0067DD94F84D30002B40F09A801D4E357867
:1013AC00002DBFD01C4B1B78002BBBD10B78002B16
:1013BC00B8D094F85030AB4200F09180052D84F8F1
:1013CC00505040F29780012384F84E30AAE7012A4E
:1013DC0078D0022A70D0032AA4D1252DA2D10F498E
:1013EC00B4F84A2094F84C008854002384F8483010
:1013FC0098E700BF3407002020070020C803002016
:10140C00C0030020B00600207C060020C10600208E
:10141C00AA060020DC06002064060020000500203F
:10142C00019303F01BFD019B6E4918B394F8442003
:10143C000132D2B2642A84F844201BD901221A70DA
:10144C00D4E90173059363690493A3690393E36976
:10145C000293236AE66A0193D4E903EAD4E909B555
:10146C0067E76B1E2E2B16D85F4B604E1A80EDB2C1
:10147C00357097E7D4E90172059262690492A2690A
:10148C000392E2690292226AE66A0192D4E903EAC3
:10149C00D4E909B53AE7002D80D194F84F30524980
:1014AC00524A012B4FF0000308BF84F84D500B80BB
:1014BC00137084F84E3035E7032384F84C5084F8CD
:1014CC0048302FE70223A4F84A5084F8483029E723
:1014DC004549464B0D801A7084F84E2022E7052DA5
:1014EC0008D994F84E300133DBB2052B84F84E301A
:1014FC007FF618AF0023013D84F84E30232D16D80B
:10150C00DFE805F0126C6864605C554E4A46153E87
:10151C00322B1515151515241F1515151515151523
:10152C00151515151515151B314B01221A70314A5D
:10153C003178117000233370F4E6012384F84830BD
:10154C00F5E72D4A2D4B527C1A70F0E72A4B2B4AAB
:10155C005B7CC3F101031370E9E70022012384F8DB
:10156C00512084F85330E2E794F84F300122934233
:10157C0084F8512084F85220D9D184F84D30D6E724
:10158C0000F000FC1C4B1A4A5B7C01331370CEE755
:10159C00194B01229A74CAE7174B00229A74C6E7BA
:1015AC001549164B0120002248741A70BFE71249E6
:1015BC00124B0020012248741A70B8E7104B01221C
:1015CC001A70B4E70A4B05221A70B0E7084B0422D4
:1015DC001A70ACE7064B03221A70A8E7044B0222E0
:1015EC001A70A4E77C06002066060020DC060020AA
:1015FC0082060020DD06002000050020540000209B
:10160C00C606002030B5824D95F85130002B36D1EE
:10161C0095F85230002B3DD095F85330002285F8C8
:10162C005220002B00F0C08000237A4C85F85330F8
:10163C004EF6F173012285F85E20774A774892F8CE
:10164C0000E06B6605EB8E03802200EB8E001A67C0
:10165C001146AC66043013224FF0010C0CFA02F365
:10166C002340D34083EAD111013AC901531C40F8FD
:10167C00041FF3D105EB8E050023EB6630BD95F806
:10168C005E40002C49D095F85230002285F85E203F
:10169C00002BC1D195F85330002BC5D1604B1B7872
:1016AC00002B00F08580C30B024640F0838083132F
:1016BC00012B00F0A3804313012B00F0A180031336
:1016CC00012B00F09980C312012B00F09F80831234
:1016DC00012B00F099804312012B00F09380002322
:1016EC002B66030A83EA10134340DB4303F00F031A
:1016FC0043EA021319134B4A03F00F00515C145CBC
:10170C0044EAC134C3F30321515C44EA8124C3F39A
:10171C000311525C44EA42148FE7B5F85C30B5F81B
:10172C005A20B5F8581001339BB20132013192B2F4
:10173C0089B2272BA5F85C30A5F85A20A5F85810CB
:10174C0041D8C72A4ED9384A384B1288A5F85A4086
:10175C00A3FB0232C2F3C70242F4806295F8523006
:10176C00002B7FF459AF95F85330002B7FF45CAF0E
:10177C00110A81EA12115140C9432A4801F00F01A4
:10178C00C2F3132441EA021310F804C0445CC2F300
:10179C00031102F00F02415C825C44EACC3444EA4F
:1017AC00812444EA421445E7214C4EF2010341E7FF
:1017BC004FF6FF720F21083942FA01F343EA412236
:1017CC00296690B28DE71B4B1849B3F90030A5F888
:1017DC005C4081FB0321DA17C2EB2112D2B242F436
:1017EC00C062BBE7C7297FF613AF134BA5F858406F
:1017FC001A7842F40072B1E70C21DCE70E21DAE72B
:10180C000D21D8E70921D6E70A21D4E70B21D2E72D
:10181C00C8030020FB3D0700C30300203404002054
:10182C006406002004610008A60600201F85EB5109
:10183C003B670700AC060020C206002030B5039CB5
:10184C0005468D4209DC13E0A34213D0B1EB6C0FBB
:10185C000DD0754510DC0446724601EB020C1819CC
:10186C0095424FEA6C0E4FEA6000EDDB204630BD2E
:10187C009542FBDA184630BD0EF101010346E0E754
:10188C000346401A48BFC81A704700BF04494A6A49
:10189C0080B292B24B6A9B1A9BB28342FAD37047C6
:1018AC000048014000F1FF3C58B106494A6A92B227
:1018BC004B6A9B1A9BB2B3F57A7FF9D3BCF1010C3E
:1018CC00F4D2704700480140002965D00139421E0E
:1018DC0050FA81F1002027E0C3B240B2002831DB7E
:1018EC005800C3B240B2002833DB5800C3B240B238
:1018FC00002835DB5800C3B240B2002837DB580053
:10190C00C3B240B2002839DB5800C3B240B2002841
:10191C003BDB5B00D8B25BB24000002BB8BF80F061
:10192C0007008A42C0B236D012F8013F584010F07E
:10193C00800F4FEA4000CFD080F0070358B2002848
:10194C00DBB2CDDA5B0083F0070358B20028DBB2C0
:10195C00CBDA5B0083F0070358B20028DBB2C9DA9C
:10196C005B0083F0070358B20028DBB2C7DA5B00D8
:10197C0083F0070358B20028DBB2C5DA5B0083F0B2
:10198C00070358B20028DBB2C3DA580080F0070016
:10199C0043B2C0B2C0E7704708467047026803FB09
:1019AC0003F303EB430C22EA0C0201FB03F3134396
:1019BC000360704703FB03F310B4046803FB01F1ED
:1019CC0003FB02F203EB430324EA03040C4304601D
:1019DC00C16810BC21EA03031343C360704700BF06
:1019EC0010B50C4CBDF808C0A170090A6170110A41
:1019FC00E170190A2070227161714FEA1C220921D1
:101A0C002046A371E27184F808C0FFF75DFF607295
:101A1C0010BD00BFCC04002070B50B4C0B4E04F174
:101A2C003005B64620686168A268E368F446ACE805
:101A3C000F001034AC42E646F4D104483021FFF7D5
:101A4C0043FF86F8300070BD00050020CC04002058
:101A5C00BFF34F8F0549064BCA6802F4E06213438B
:101A6C00CB60BFF34F8F00BFFDE700BF00ED00E080
:101A7C000400FA0570B5BA4CBA4D82B02968C02280
:101A8C00204603F07BFB6378022B40F21581A27990
:101A9C00511EC9B2E37D2A2B55D8181F052852D9DF
:101AAC00032B55D90A3BDBB2202B56D9237EA3F14D
:101ABC000800C0B2882858D803EB8303AA48AB4E61
:101ACC0003EB83039B00A0FB03033129A8484FEAD7
:101ADC009303B0FBF3F3F362AB804DD802EB8202BD
:101AEC00520002F5C87189B2637E2A81A3F13200DB
:101AFC00642898BFD218A37EA98103EB83034FEA15
:101B0C00C30303F1140398BF92B20220EB816A81E4
:101B1C0002F0F8F86378002B38D1E8894FF4FA73A7
:101B2C00009340F6B8324FF47A734FF49671FFF786
:101B3C0085FEA37CA5F8500013B34FF47A73C4F858
:101B4C00C83002B070BD1020032B84F8C000A9D897
:101B5C00DB00DBB203F10A00E07584F8C030237EB1
:101B6C00A3F10800C0B28828A6D9804841F2873377
:101B7C003129EB80C362B1D94FF4C8710022B3E7AD
:101B8C004FF4FA63C4F8C83002B070BDA07F0B28C4
:101B9C0088BF052002F0B6F894F8213094F8202084
:101BAC0094F8221094F82300A87503F26B335B00B1
:101BBC006B8294F82830053B142B84BF052384F8E2
:101BCC00283094F8293002F27712013B5200092B8D
:101BDC002A8294F8252088BF0A2302F1FA0288BFD2
:101BEC0084F8293094F82A302A83002284F827209C
:101BFC005A1E01F25E51082AA98269D90A2384F877
:101C0C002A3094F82B30617AE27AA07AA862463BAB
:101C1C00462B84BFFF2384F82B3094F82C30013BE7
:101C2C00622B9CBF012384F8C13094F82D30013B0A
:101C3C00092B84BF052384F82D3094F82E304900ED
:101C4C005200092B6962EA6206D8042B0CD8DFE833
:101C5C0003F003817D0B7400464A0023012184F8B4
:101C6C00C23084F8C33011706379092B49D809222A
:101C7C0084F8C42085F8483085F8493085F84A3016
:101C8C00E8893D4AE17EB0F5967F3CBF002385F89C
:101C9C004B302023B3FBF1F1A2FB0032324B520943
:101CAC00B2FBF1F2A5F84C20A3FB0023DB08B3FB3D
:101CBC00F1F3A5F84E3031E7304AC4F80520002185
:101CCC004FF06413C4F80930C4F80D100122E1E69A
:101CDC00C3EB4312C3EB82035B006A8923492E3B9F
:101CEC00DBB21A446A812A89AB761A442A81AA8B00
:101CFC001A44AA83AA891A44AA814A6C13434B64D6
:101D0C007FE7002284F8C42095F84810A2F1333202
:101D1C00A2FB0323DA08B1EBD30F88BF85F8482068
:101D2C0095F849309A4238BF85F8492095F84A30E1
:101D3C009A4238BF85F84A20A2E711490D4A01237F
:101D4C000B700021117084F8C2308DE7012384F8E8
:101D5C00C33089E7074A012384F8C230137083E744
:101D6C000005002000000020ABAAAAAA002C01400C
:101D7C00F0821E00150400201F85EB51A001000A03
:101D8C0017040020024B03481A68C02103F09AB9CB
:101D9C00000000200005002038B5294C94F8543080
:101DAC00012B3DD094F85530264D5A1E12F0FF02EF
:101DBC0024D084F8552003F0010384F8523072B615
:101DCC0095F83F313BB362B603F054F9D5F8C830FF
:101DDC00D5F84021A16D03F5FA7393423CBF012362
:101DEC0084F8563094F8553005EB4303002285F8FF
:101DFC003C2185F84421A3F8461138BD0123062265
:101E0C0084F8552085F83E3184F8523072B695F836
:101E1C003F31002BD7D194F8550003F08DFCD2E75D
:101E2C0094F85520074D0132D2B2062A99BF84F896
:101E3C00552002F0010384F8553085F83E31BCE79B
:101E4C0000000020000500201C4AD36823F0010389
:101E5C0010B51B4CD360FFF79FFF1A49B4F856011D
:101E6C00B4F854218B6D024403EB520394F82F20E9
:101E7C0058088865C2B994F8C02000FB02F2C2F37E
:101E8C008F1291F85610A4F85A21C2EB9303A4F8C0
:101E9C005C3181B1D4F8603142F20F7293429CBF35
:101EAC000133C4F8603110BD94F8582100FB02F2E4
:101EBC00C2F38F12E5E703F0D5F8EBE700440140DD
:101ECC00000500200000002038B5174D95F85C3057
:101EDC0073B1002403E095F85C30A34208DD03F0F5
:101EEC00ADF895F85230834204F10104F3D138BDBA
:101EFC0072B603F0ABF80D4A0D48B2F85C11446AA7
:101F0C00B2F856510B4BA2F85451A2F8564101317C
:101F1C00002242625A62D9621A61DA6842F0010206
:101F2C00DA6062B638BD00BF00000020000500205A
:101F3C00001000400044014070B5C84CA37C82B036
:101F4C007BB394F8C230002B00F09080C44D94F811
:101F5C002630002B40F06481B4F86621B2F5836F13
:101F6C0080F09782A2F130039BB2B3F57A7F10D246
:101F7C00617C95F85460C1F10100864200F02D831C
:101F8C0095F85D105B009BB2C1F12F010B44A4F8D6
:101F9C0068312F2A0AD80023A4F8683184F86F31ED
:101FAC0004E0B4F86631AE4DA4F8683194F87021B1
:101FBC0095F85E309A4203D9A37D002B40F0E38064
:101FCC00E67CAEB3B4F868011D2800F2C78000238C
:101FDC00A4F8723194F8283003EB8303B0EB830F31
:101FEC004FEA830180F2C68094F86E31002B40F0EA
:101FFC00AE8094F87C31002B00F0A980E27CB4F820
:10200C00720150232E2113FB02138342C0F22C8148
:10201C0094F88231002B00F0C981013B042B00F2B3
:10202C00C281DFE813F0BE019D039A039703BE0142
:10203C0094F87431002B00F08C8094F87531002BDF
:10204C0040F06681D4F878218649D31781FB0212BF
:10205C00C3EB22339BB2B3F5006FA4F87231C0F01E
:10206C00DB8140F2FF73A4F87231BDE794F82620AF
:10207C007B4DB4F86601002A00F09080AE7D7600AE
:10208C0006F57A7188421CDD667C95F85420B242C4
:10209C0000F03D8394F83F31002B40F0BB800023CF
:1020AC0084F86A3140F2FF7300934FF4FA622F23E5
:1020BC00FFF7C4FBAE7D0346B4F86601A4F86831A3
:1020CC007600C6F57A72824221DD637C95F8546005
:1020DC00C3F101018E4200F0DD8294F83F31002BF8
:1020EC0040F098802F230021009340F2FF7384F876
:1020FC006A11FFF7A3FBAE7D03467600B4F86601C8
:10210C00A4F86831C6F57A739842C0F2838006F55C
:10211C007A76B0427EDC94F83F210023A4F8683133
:10212C00002A77D0012284F83F3184F86A2171E0CB
:10213C00E17C2E22502313FB0123B4F8722193422D
:10214C00BFF666AF94F83F61002E00F0C28102B07A
:10215C0070BDB4F86831A4F8723145E71E283FF41D
:10216C0039AF94F8282002EB82029200904211467B
:10217C00C0F2ED8040F2FF720092A023FFF75EFBED
:10218C00A4F8720130E703F099FA02F05FFF002225
:10219C006623A4F8722184F8703125E7AA7D5200D9
:1021AC0002F57A71884240F38981637C95F854205A
:1021BC009A4200F04F8240F2FF7300934FF4FA62A0
:1021CC002F23FFF73BFBAB7D02465B00B4F86601A7
:1021DC00A4F86821C3F57A72824240F3F881637CDB
:1021EC0095F85460C3F101018E4200F074822F23E4
:1021FC000093002140F2FF73FFF720FBAB7D0246FA
:10220C005B00B4F86601A4F86821C3F57A729042B9
:10221C0080F2DD8194F8C230002B3FF4C7AE96E615
:10222C00B4F86631B3F5836FC0F09D80617C95F88E
:10223C0054208A4200F07D8294F83F21002A7FF4DA
:10224C00B5AE95F85D206FF40060C2EB430300213E
:10225C00034484F86A11A4F86831A7E6000500204D
:10226C0000000020AD8BDB6894F86431002B00F08B
:10227C003F81002A00F030812B894FF4FA620092E2
:10228C00283340F2FF728921FFF7D8FAA4F88001B5
:10229C0094F82630002B7FF44BAFE07CB4F872112D
:1022AC0084F83F3150222E2312FB003399427FF7E2
:1022BC00AFAE2E2907D9627F1E231341D4F86021BB
:1022CC00934200F26181B4F88031B5F892209A42C1
:1022DC003CBFA4F88021134694F8C12032B1B5F963
:1022EC0094209342C4BF93B2A4F88031D4F88C21CB
:1022FC00002A7FF72CAF2F297FF629AFC548D117BD
:10230C0080FB0202C1EB22321344A4F880311EE799
:10231C00D5E91832B4F8680100922F2140F2FF720F
:10232C00FFF78CFAB4F86821BB4B93FBF0F3E07E1B
:10233C002E2A4FEA500093FBF0F3A4F876313FF6C7
:10234C0081AEA4F87261AE66C4F878614CE6A02345
:10235C0000931E212F23FFF771FA0346A4F8723164
:10236C00B4F8680136E6303B9BB2B3F57A7F80F067
:10237C008280627C95F85400C2F10101884200F021
:10238C009A8194F83F21002A7FF410AE95F85D20D5
:10239C00C2EB430300212F3384F86A11A4F868318F
:1023AC0004E601F0EDFD002384F88231237D002B3F
:1023BC0039D194F86421A4F88031002A00F0F3801C
:1023CC0094F82630002B3FF4BDAE94F83F31002B2F
:1023DC007FD094F8C230002B00F0F581B4F8661170
:1023EC00A1F130039AB2B2F57A7F80F00D8295F8A4
:1023FC005D30C3EB42032F339BB2A4F8843140F21F
:10240C00CE72934240F2DC8103F02EFB94F83F61D4
:10241C00002E7FF49CAE5CE02F2B3FF6E5AD302315
:10242C00A4F87231E0E594F86431002B73D1267F67
:10243C00C4F86031012285F8562084F83D31002E15
:10244C0067D0E17C002967D1012E65D194F8293041
:10245C0003EB830303EB8303DB009BB240F2CE72EE
:10246C009342A4F8843140F2E18103F0FDFAE17C5F
:10247C0094F83F6152E094F83F210023A4F86831AE
:10248C00002A3FF493AD012284F83F3184F86A218D
:10249C008CE5637C95F85410994200F0BF8095F858
:1024AC005D00A2F58361490089B2C0F12F00A2F151
:1024BC00300301449BB2A4F8681156E5C2F57A7258
:1024CC009042FFF68CAE0023A4F8683184F86F318B
:1024DC00A0E6B4F87211ECE64FF4FA6200922B8984
:1024EC0040F2FF722F21FFF7A9F9A4F88001CFE683
:1024FC0003F0E4F895F85630002B00F058816B8906
:10250C00E27CB4F87201A4F87E31012184F86411E4
:10251C00AFE603F0D3F8E17C94F83F6195F85530C1
:10252C00013BC3EB0312B5F8903003EB82031AB2F4
:10253C00B2F5B47F9BB2A6BFA3F5B4739BB2A4F85B
:10254C00862103F1770212B2A8BFA4F88631B2F546
:10255C00B47FA8BFA3F1F102A4F8882103F1EF0224
:10256C0012B2B2F5B47FA6BF793BA4F88A31A4F8B5
:10257C008A210023012908BF84F86E11A4F8803148
:10258C00002E7FF4E4ADA4E7B4F880316A8993425D
:10259C003CBFA4F880211346AA899A423CBFA4F8F8
:1025AC008021134691E6237FC4F86021012185F830
:1025BC005610002B40F0018194F83F31002B00F0B5
:1025CC00138194F82630002B7FF403AFBFE503F59D
:1025DC007A738342FFF61EAE75E7B5F85020AB6DEB
:1025EC009A4280F0C080B4F86C31C72B00F2BB80EB
:1025FC000123002685F85630C4F8606185F8541024
:10260C0002F024FDB4F8662184F86F61A2F1300366
:10261C00B6E400BFAD8BDB6800879303B5F85010B0
:10262C00AA6D914280F0B180B4F86C21C72A00F2F7
:10263C00AC800122C3F10103002685F8562085F8F1
:10264C005430C4F8606102F001FDB4F8662184F8DE
:10265C006F6124E7B5F85000AA6D904280F08B8032
:10266C00B4F86C21C72A00F28680C3F1010300265E
:10267C00012285F85430C4F8606185F8562002F0C8
:10268C00E5FCA97DB4F8660184F86F61490001F599
:10269C007A7190E594F86A6100214FF0010CA4F86E
:1026AC00681184F83FC1002E3FF4B4AD85F8543066
:1026BC0084F83F1116E594F86A0100210126A4F86C
:1026CC00681184F83F6100283FF470AC85F8542001
:1026DC0084F83F115AE6B5F85000A96D88425DD2D6
:1026EC00B4F86C11C72959D80122002685F8562058
:1026FC00C4F8606185F8543002F0A8FCAA7DB4F8E7
:10270C00660184F86F615200C2F57A726FE594F835
:10271C006A61A4F868314FF0010C84F83FC1002EB7
:10272C003FF478ADACEB020284F83F3185F85420CD
:10273C00B5E494F86A0100210126A4F8681184F824
:10274C003F6100283FF432ACB21A85F8542084F86B
:10275C003F1176E501F0A6FB25E601F071FC22E6BF
:10276C0001F03EFC1FE694F86E31002B7FF440AF75
:10277C00A4F866310FE494F86E21002A7FF475AF4B
:10278C004FF47A70A4F8660115E594F86E21002ACE
:10279C007FF44FAFA4F86621FFF7FDBB94F86E11E0
:1027AC000029A1D14FF47A70A4F866011FE594F8C2
:1027BC006431E3B102F056FCA1E603F055F9FFE5F4
:1027CC0002F044FFBEE4B4F866114FF47A70FFF7E0
:1027DC0057F894F8C22000F57A739BB2A4F88431B0
:1027EC00002A3FF40CAEF9E502F068FFE8E5FFF7CC
:1027FC00D3FA114B42F2107141F28832A9655A6238
:10280C00012384F86431D5E7B1F5836F38BFB4F890
:10281C008431FFF4F4AD95F85D306FF40062C3EBD6
:10282C00410313449BB2A4F88431E8E502F00EFF97
:10283C00E17C84F83F6171E60010004010B50E4C4D
:10284C0094F89031012B0DD0022B03D0BDE8104031
:10285C00FFF772BBB4F89401FEF7D4FE002384F8A2
:10286C00903110BDFEF766FC002384F89031BDE872
:10287C001040FFF761BB00BF00050020F8B54F4EBC
:10288C004F4F96F85410002977D1B7F886310133A1
:10289C001AB2B7F888310133B2F5B47F1BB2B2BFAC
:1028AC00A7F88621A7F886110A46B3F5B47FA8BF0E
:1028BC000023A7F88831B7F88A3101331BB2B3F57E
:1028CC00B47F77DAA7F88A3106EB4202B6F86813C0
:1028DC00B2F99830B0883B4D3B4C0B4400FB03F3F2
:1028EC0085FB0312D81797F82D30C0EBE21003FBD1
:1028FC0000F0C31784FB0020C3EBA00080B202F0F1
:10290C0007FEB7F98831B6F8680306EB4303B3F951
:10291C00982097F82D300244B08800FB02F285FB1A
:10292C000201D017C0EBE11003FB00F084FB002385
:10293C00C017C0EBA30080B202F0F0FDB7F98A31EA
:10294C00B6F8680397F82D2006EB4303B3F99830DB
:10295C000344B08800FB03F385FB0315D817C0EBC9
:10296C00E51002FB00F084FB0034C017C0EBA400A0
:10297C0080B2BDE8F84002F0D7BDB7F88621B7F8B1
:10298C008831013A12B2013B1BB2002AB8BF40F2A7
:10299C006712002BB8BF40F26713A7F88831B7F85D
:1029AC008A31A7F88621013B1BB2002BB8BF40F23D
:1029BC00671387E70023A7F88A3185E7000000201A
:1029CC0000050020D34D62106766666638B5254D4C
:1029DC002549AB6D4A6A254C03EB430313FA82F38A
:1029EC00A4F8562100224A6294F8C020980800FBF3
:1029FC0002F2C2F38F12C2EBD303A4F85A21D4F81B
:102A0C006021A8659BB2042AA4F85C3127D94A6AD4
:102A1C009A42FCD3FFF7C0F9D4F86031607F94F888
:102A2C0026100022013384F83C2184F83D2150EA21
:102A3C000102C4F8603105D1D4F8C830AA6D9A42AD
:102A4C0006D338BD132BFCD9AB6DB3F5FA6FF8D8A0
:102A5C00002385F85630BDE8384002F003BB4B6AC2
:102A6C00D8E700BF00000020001000400005002047
:102A7C00F8B5914CB4F89801B4F89A31B4F89C11AB
:102A8C00B4F89E21B4F88051A4F86C510130013394
:102A9C00A4F89801A4F89A3194F8A00194F87C3128
:102AAC00013101320343A4F89C11A4F89E2141D1B9
:102ABC0094F8A121002A3DD0B4F86851002D40F0C3
:102ACC00D281B4F8A23101339BB244F620618B421F
:102ADC00A4F8A2312ED9B4F8A4311E2B40F24F82A7
:102AEC0094F8243001218B4284F87C1140F04C8204
:102AFC00B4F8A61171484B08A0FB0323DB09B1F510
:102B0C00B97F84F8A0310DD36D4F4AF6AA2601F097
:102B1C0001FA6420FEF7C6FE94F8A0313E60013540
:102B2C00AB42F4DC94F8C33094F8C220134301D1C7
:102B3C0084F82630E17F79B1624BB4F8A82193F880
:102B4C006A33013B01320B4492B203EB8303B2EBC9
:102B5C00830FA4F8A8217ADC94F86E61002E51D171
:102B6C00584D95F8563023B194F86431002B40F051
:102B7C004281B4F89E31142B19D994F8C13001213B
:102B8C00002284F8AB11A4F89E21002B00F0A08049
:102B9C0094F86431002B40F07D81637F3BB994F84D
:102BAC00743123B194F86431002B40F0E28094F836
:102BBC00C430B4F89C219A422AD8B4F87E21A4F8E7
:102BCC006C2194F87C311BB194F86411002954D118
:102BDC0094F83F11002941D0E988B4F884313A487F
:102BEC0001FB03F380FB0350DB17A3EBE0130B4457
:102BFC009BB2A4F8AE313548A4F87E21C0E90D3360
:102C0C00C162C363B4F8B0310133A4F8B031F8BD7C
:102C1C00D4F86031B4F87E110022952BA4F89C21D5
:102C2C003BD895F84830DBB285F89833B4F86C2172
:102C3C00501A984203DDCA1892B2A4F86C21881A73
:102C4C008342BEDACB1A9AB2A4F86C21B9E70122FE
:102C5C00002384F8AA21A4F8A8317DE7207F02285C
:102C6C0000F0EA80E988184801FB02F3A0FB03039B
:102C7C00C3F3CF13A4F8AE31BDE7B4F872112F290A
:102C8C00A6D9E988104801FB02F3A0FB0303DB097A
:102C9C0001339BB2A4F8AE31ADE79529C1D9D4F874
:102CAC004031B3F5FA7F8CBF95F8493095F84A302E
:102CBC00DBB285F89833B9E700050020B9D31FB112
:102CCC000030004000000020D34D6210002C014069
:102CDC00637F002B3FF463AF94F86431002B3FF417
:102CEC0066AFAB6DB5F86E23D5F88013D5F87803C5
:102CFC009A1AD5F89033C5F8702300FB021199424B
:102D0C00C5F88013C4BF1946C5F880335B428B42AB
:102D1C00C4BF1946C5F88033D5F88833D5F87C0381
:102D2C00C5F88823D31A00FB03F3D5F87403C5F850
:102D3C00843300FB0233D5F894230B449342C5F83B
:102D4C008C33C4BF1346C5F88C2352429A42D4F834
:102D5C008C11C4BFC5F88C2313468E4A0B44934286
:102D6C0040F30181C4F88C2194F87431002B3FF4AA
:102D7C001EAFD4F89431B4F87621A96F286F9A1A43
:102D8C00D5F88830AA6600FB02119942A967C4BF26
:102D9C001946AB675B428B42C4BF1946AB67D5F88B
:102DAC008030686FC5F88020D31A00FB03F3E86EFF
:102DBC00EB6700FB0233D5F88C200B449342C5F82B
:102DCC008430C4BF1346C5F8842052429A42D4F8CA
:102DDC007811C4BFC5F8842013466F4A0B44934244
:102DEC0040F3C780C4F87821D4F86031632B9CBFC2
:102DFC000023AB67DBE602F029F902F01FF995F826
:102E0C0052309BBB002800F0938094F83C31013386
:102E1C0084F83C3194F84431002B7FF4AAAE94F83A
:102E2C003C2195F86C339A427FF6A3AE012384F8CB
:102E3C004431FFF7CBFD9CE6002B3FF413AF02F0BF
:102E4C007BFCE988237B554A01FB03F3A2FB03239C
:102E5C00DB0903EB83035B003C339BB2B4F86C21BE
:102E6C00A4F8AE31C7E6A4F8A23163E600286DD110
:102E7C0094F83C31013384F83C3194F84431002B04
:102E8C007FF477AE94F83C2195F86B339A427FF639
:102E9C0070AECBE794F82C20B4F9AC31296BA86A4E
:102EAC0002EB820202EB8202A3EBC2022B6C2A62BF
:102EBC0000FB021199422963C4BF19462B635B4284
:102ECC008B42C4BF19462B63AB6BE86AAA63D31A57
:102EDC0000FB03F3686A6B6300FB02336A6C0B4400
:102EEC009342EB63C4BF1346EA6352429A422C49A5
:102EFC00C4BFEA631346DA1781FB0313C2EB233218
:102F0C00B5F8943029899B1A1BB28B42A5F89430E2
:102F1C00BCBF0BB2A5F89430B3F5FA6F03DD4FF4D8
:102F2C00FA63A5F89430637F002B7FF4DAAE1BE7CD
:102F3C0094F83D3195F853200133DBB29A4284F872
:102F4C003D31BFF467AF84F83C0112E694F83D3193
:102F5C0095F853200133DBB29A4284F83D318CD280
:102F6C0084F83C6105E6002B11DC0023C4F88C319D
:102F7C00FAE6002BB8BF0023C4F8783134E784F8A4
:102F8C00A151A4F8A251D5E500F0C4FFCAE5C4F8DC
:102F9C008C31E9E660E31600F0583801D34D62102D
:102FAC00AD8BDB682DE9F04F85B002F01BF94FF4C7
:102FBC007063B44AD3F8E010914205D1B24AD3F809
:102FCC00E410914200F0F983B04DB14C02F0E6F9F7
:102FDC0002F0C0FAFEF74EFDE378022B03D1237901
:102FEC00142B00F0228441F202410323A4F80310B5
:102FFC002A68A7486370C02102F064F8637C227DC4
:10300C00A988E980013B18BF012385F8543002B927
:10301C00E27494F82630A3B12989B5F89A236B8908
:10302C00323101204FF47A76298132323233002149
:10303C00AE8385F84B00C4F81200A175A5F89A234D
:10304C006B8100F0EDFE0023A4F8A43102F008F926
:10305C00904B4AF6AA221A6001F07CFE94F8753166
:10306C0013B1012384F8743101F000FF894FDFF8AC
:10307C002892DFF82882DFF828A24AF6AA26B4F8AC
:10308C004A11B4F84831B4F84C21B4F84E010B4451
:10309C001344B4F85011B4F8522103440B441344B4
:1030AC00D4F8602104335B10042AC4F8943100F284
:1030BC00DD81A37C002B00F05F82042385F86B3349
:1030CC0085F86C33637D3E60012B00F0D981022BB7
:1030DC0000F0E381B4F8B03142F21072934209D996
:1030EC0094F87C11002940F04F8349F640429342FA
:1030FC0000F27083B4F8982144F620639A4210D9F8
:10310C00B4F9AC31D4F8B4211B0489FB0301194484
:10311C00DB17C3EB212313440022C4F8B431A4F809
:10312C009821D4F86021B2F57A7F40F2C981002150
:10313C00B4F8683184F87011C72B40F22382E17C1B
:10314C0011B19F2B40F2C78194F8B811002900F0FF
:10315C00B081B3F5C87FC0F0C581D4F8943194F830
:10316C003E0188FB03C1A1EBE371C4F8401110B11F
:10317C000A2A00F2258294F8C131002B00F09A80C3
:10318C00AB6D322B40F29680464B1022002183F817
:10319C000B1383F8152383F80C2394F8AAB1BBF115
:1031AC00000F40F0968094F8C631002B40F0EE8171
:1031BC0094F8ABB1BBF1010F00F0A58094F86E311F
:1031CC004FF0000B84F8D7B1002B40F01C8194F821
:1031DC006431354AD4F89411344892FBF1F213FB64
:1031EC0002F39BB2A0FB032095F84B20A4F8C4314A
:1031FC00C008A4F8D801002A40F01E824FF4FA63EC
:10320C00A5F8923094F82B1094F8C2018142C0F0CA
:10321C000682D4F86031632B00F28A81AB6DB3F572
:10322C00FA7F40F285810C2385F85C3094F82F30BE
:10323C00002B40F094811E4A526A4AF6C8739A4297
:10324C007FF61DAF94F864B1BBF1010F7FF417AF9B
:10325C0094F87031013384F8703101F0F7FEB4F852
:10326C00723185F856B02F2B05D8002384F86431C1
:10327C0041F28833AB650023C4F86031FFF7A6FB3D
:10328C00FDE600BFDAE32559D963B84E00000020F3
:10329C000005002000300040B7600BB65655555560
:1032AC001F85EB5100E100E0C0270900CDCCCCCC50
:1032BC0000100040BC4B0022102183F80B1383F844
:1032CC00152383F80C2394F8AAB1BBF1000F3FF43B
:1032DC006AAFB4F9B631B4F8C411B4F8AC2194F8AF
:1032EC00C20100919BB2B4F8A611FEF779FB0A203B
:1032FC0002F04EFC94F8ABB10023BBF1010F84F843
:10330C00AA317FF45BAF01F06FFC5946A74801F07E
:10331C0019F8B4F8C80101F007FDB4F8CC21A44B9E
:10332C00A4F8CA0140F6E44101FB02F2A3FB02132C
:10333C00D21A03EB5203B5F89C2384F8C201DB0AC2
:10334C0094F8D000B4F838E102FB03F3B4F8A621EA
:10335C00AAFB031304EB400CC2EBC20202EB5312A8
:10336C000130D4F8CC30BCF8D4B0ACF8D4E0C0B256
:10337C003128734488BF0020A3EB0B0384F8D000E2
:10338C00C4F8CC30AAFB03031B0940F6E440A4F8B4
:10339C003A319BB2C4F8D03100FB03F38548A0FB53
:1033AC00030343F30F23002BB8BF0023A4F8AC3165
:1033BC0094F82430D110012BC2F3CF02A4F8A6212B
:1033CC0000F07781022B08D1237A934240F27A8164
:1033DC00B4F8D4310133A4F8D43194F86E31764872
:1033EC00B4F8D41142F2107200FB0322914200F3A4
:1033FC00718100224FF0000B84F8AB2184F8D7B117
:10340C00002B3FF4E4AEB4F87231302B72D994F83F
:10341C007C21002A6ED0313B572B00F27A8194F834
:10342C00DA31002B40F0F081FFF728FA94F81BE01A
:10343C00B4F872017822302141F6583340F22A3C1C
:10344C00B3FBFEF3BCFBFEFCCDF800C0FEF7F6F9B7
:10345C00A5F8A00380B2FEF719FAB5F8A0234FF433
:10346C001673B3FBF2F3A4F8C43108E6032385F812
:10347C006B3385F86C33637D3E60012B7FF427AE94
:10348C00AB880093A86D5B08C8226021FEF7D6F9C3
:10349C00637DE880022B7FF41DAED4F84031A3F19C
:1034AC006502942A3DD803EB430203EB8203EB80C5
:1034BC0010E6952B94BF64230A2385F85E304CE606
:1034CC00B4F8683193B9642A84F870315AD8E17C25
:1034DC0000293FF439AE002184F8701194F8B8112A
:1034EC000029E6D0002384F8703136E6642A7FF692
:1034FC0026AE21E694F81CB001239B4584F8DA3102
:10350C0000F0A780BBF1020F00F0BF802B4B002214
:10351C00C3E90D22DA6302F0D1F80023A4F8C43118
:10352C00ADE5013B622B39D840F21453EB80D1E569
:10353C000C230093D4F8400103234FF4FA72642156
:10354C00FEF77CF9AB6D85F85C00312B9CBF022338
:10355C0085F85C3094F82F30002B3FF46CAE1723B9
:10356C000093B4F86C010D234FF4FA626421FEF75A
:10357C0065F984F858015EE6062385F86B3385F807
:10358C006C339FE5002184F87011D8E5FEF744FAFE
:10359C00312002F0FDFA84F8C6B109E6F82B84BF9D
:1035AC0040F6B243EB8095E500E100E000240140D9
:1035BC0001011000FF04EC4F54D9FFFF002C014017
:1035CC00D4F8BC01FEF75CF9D4F84031B0EB530FE2
:1035DC001AD9B3F5FA6F17D294F8C021013284F8D6
:1035EC00C021A27C0021C4F860119AB9B4F87221F0
:1035FC002F2A0FD9002284F864216A895208A4F872
:10360C007E21012285F85620002284F83E21C4F840
:10361C00BC31B0E5AA6DB2F57A7FEED9EAE7B5F820
:10362C009E33012200925B0801F10A020A39FEF76F
:10363C0005F9A5F89200ECE5B5F89E330093AB8B39
:10364C00B5F84E20B5F84C10FEF7F8F8A5F8920036
:10365C00D8E594F82930EA887B4903EB830303EB24
:10366C008303DB009BB2A4F8843102FB03F381FBE0
:10367C000301DB17A3EBE11313449BB2632BA4F8F8
:10368C00AE313BD802F0F0F947E7584602F054F857
:10369C00EA88237B02FB03F36B4AA2FB0323DB09BF
:1036AC0003EB8303694A5B003C33C2E90D33D363FC
:1036BC0033E794F8A0312A8B89B202FB03F38B42D7
:1036CC003FF786AE94F8D631002B7FF486AEA4F883
:1036DC00D43182E64FF0000B012384F8D631A4F8E4
:1036EC0072B101F0EBFF01F0B1FC94F86E3184F88B
:1036FC0064B1A4F8A4B184F87CB17AE601F0A6FF19
:10370C00524BB4F8AE2184F83FB1C3E90D22DA6311
:10371C0003E7012384F8DA31FFF7B0F8B4F872311B
:10372C00C82B04D95023A4F886B1A5F8A033B5F85A
:10373C00A003FEF7ABF8B4F98631002B7FF49FACF5
:10374C00434984F86E31012284F83F3142F2283328
:10375C00AB65C4F84031C4F8BC3185F856204B62D7
:10376C0084F86421637F95F8A22385F855201422F0
:10377C00C4F860211BB1B5F89A33A4F87E31FEF77A
:10378C000BFB01F0D7FE7AE401F098FF2F4B0025DC
:10379C00C3E90D55DD6384F87C51A4F8725184F8AB
:1037AC00A151A4F8A45101F0CDFE2A484FF4807227
:1037BC00294602F08DFCFEF74BF993F8EC30264DC0
:1037CC002B2B3CD0352B36D01F2B04BF234B2B601F
:1037DC00FFF7FBBB039101F071FF03991B4B84F8BE
:1037EC007C11C3E90D11D963A4F8721184F8A111ED
:1037FC00A4F8A411039101F0A5FE039915484FF408
:10380C00807202F065FCD6E7154AD36823F00103F9
:10381C00D36001F01BFC0D4BC3E90DBBC3F83CB0EE
:10382C0002F060F984F8DAB1FEE56378022B3FF61A
:10383C00E5ABFFF7D8BB0B4B2B60FFF7C6BB0A4BB6
:10384C002B60FFF7C2BB00BFD34D6210002C0140B0
:10385C00001000403407002000000020007C00080D
:10386C000044014000F8000800F80108F0B5604C75
:10387C00D4E90002101A6FF4487240F276538218A1
:10388C009A4283B02AD85B4E5B4D002333802B7851
:10389C00002B3CD06B780146ABB9AB78002B00F019
:1038AC008E80A888554F01333988AB70FDF7E8FF3F
:1038BC00322866D900223B882A706A78AB804AB1DC
:1038CC00D4E90031C91A40F2E14399424DD9AB79A0
:1038DC004B2B77D80023A868338004E04649484B2B
:1038EC00886800221A804749474A0B881268A0EB67
:1038FC00030C944503DD13440B8003B0F0BD1C1A7C
:10390C00A242BABF9B1A0B80088003B0F0BD3F4A9D
:10391C00947C74B13E4A128890421AD83D494FF4B7
:10392C007A7409880094FDF789FFA860002333801E
:10393C00D9E7324B1A88374B198840F2FF73009342
:10394C002F23FDF77BFF3028CEBFA860AC6020464C
:10395C00ECE72A4B511C1A884FF4FA63009340F29F
:10396C00E933FDF76BFFA860E0E72A48AB790288E2
:10397C00C2EBC20201331144DBB2C908AB71018046
:10398C00A6E73B886268C3EBC3012368D31AAA7805
:10399C000B44C3F3CF03322A3B808ED9193B9BB225
:1039AC003B80A3F2D663194A03EBD3735B1082F806
:1039BC00213001236B7000F0E3FA3B887DE780B285
:1039CC00A8806FE7134A1149138819339BB21380EF
:1039DC00A3F2EE2303EBD3735B10002481F82030A9
:1039EC002C70FEF7CFF9AC7100F0FAFA72E700BF59
:1039FC0034070020B0060020080700201200002029
:103A0C00A406002066060020B80300200005002054
:103A1C001400002010000020514BF0B5514F1968D4
:103A2C00002544F6206E1A46A7F804E003F178044A
:103A3C00AC462E4652F8043F8B42A3EB01001946CC
:103A4C0006D070453CBF1FFA80FE01268444012538
:103A5C009442EFD1002E3ED0A7F804E0424A4348EE
:103A6C00FDB113784FEA5C15012BC56045D0404C75
:103A7C002378012B32D011780B4311D10EF1FF3189
:103A8C00022945D83B2D0BD83A493B4C0B700123EE
:103A9C003A4913700E22227020220374BA710B70F3
:103AAC00F0BD1378C560012BE1D10EF1FF33022B71
:103ABC0048D9AEF10403042BD9D801231370032287
:103ACC002D4902742B4C2D4A23700720087013705B
:103ADC002021B971F0BD44F6206EBFE7AEF1C902EA
:103AEC0092B244F656518A42DAD82249234A1370CC
:103AFC00772008700221B971F0BD0EF1FF33022B53
:103B0C0019D83B2D1ED91A4C2378012BB3D1F0BDFB
:103B1C00AEF10403042B02D8632DC1D8CDE7AEF16E
:103B2C00C9039BB244F656529342B9D801231149AA
:103B3C00124A2370DBE7AEF10403042B97D8632DF4
:103B4C00E1D8BAE70D4E0B4C0B49012333700374CB
:103B5C001370002323700E230B702023BB7186E798
:103B6C0034070020B8030020C205002008070020FD
:103B7C00C3050020C2030020C3030020A1060020BF
:103B8C0070B5524C237813B1514B1B7833B9514B50
:103B9C001B78002B6ED0012B0AD070BD4E4B1B78BE
:103BAC00002B54D001F0D6F84C4B02221A7070BD89
:103BBC00474B1B78002B50D1494D2B78012B75D0DE
:103BCC00484B1B78012B68D02378002BE5D12B7840
:103BDC00EBB1454A537C072B19D844490988052970
:103BEC0015D94348C16F00680133091A5069DBB21B
:103BFC0010FA81F1082B5374516108D1C1F3CF0332
:103C0C003C48C1F3CF115C18591A048111833A4C0A
:103C1C002088002838D0394BDD79002DBDD1334AAE
:103C2C0040F2DC5398421580B7D92F4E718BFDF7BB
:103C3C0027FE322848D8337F0133DBB2322B33775F
:103C4C0002D97578002D3BD02388738370BD01F0A9
:103C5C00BBF8224B01221A7070BD1F4B1B787BB135
:103C6C00274B1888FDF7CEFCFDF764FABDE87040D1
:103C7C0001F070B8FFF7D0FEBDE8704001F06AB8F3
:103C8C00BDE8704001F0A0B8174B1B78002BC2D1D7
:103C9C00164A13880133138070BD01F0DFF8154B01
:103CAC0048B103229A7101F055F88DE7FDF742FAFD
:103CBC0001F050F884E702229A71FFF7D7FDF2E782
:103CCC0000F0BEF9012333703577BDE77C06002088
:103CDC00C1060020A106002030070020900600201D
:103CEC00C2050020C305002008070020A406002000
:103CFC0034070020B80300206806002000050020CF
:103D0C00940600200B28034B28BF0B204000187092
:103D1C00704700BF250700202DE9F84F354C364E73
:103D2C00DFF8D880032001F007FD04F17C070023A5
:103D3C0018E094F835503249DFF8C8B0C3EBC31023
:103D4C00F7224FF47A6A0CEB400080B212FB05A20A
:103D5C004DBBC1E90D55CD63FDF7A4FD2B460234D7
:103D6C00A74211D094F834C04FF000094AF6AA22A9
:103D7C00BCF1FF0FC8F80020A6F80090D9D102348E
:103D8C000133A742DBB2EDD101F098FC1E481C4A6E
:103D9C0000881A4900239362D0624AF6AA22338023
:103DAC000A60BDE8F88FBBFBF2FA4FF00A0E174A17
:103DBC00174DB2FBFAF290B2C1F828E0C8622A782B
:103DCC0000FB02F2FE2010FB03C0124B83FB0232FD
:103DDC00114BB3FBFAFA114B0AFB00F0D20AA3FB0E
:103DEC000030C1E90D22CA63C0F34F10FDF75AFD34
:103DFC004B46B4E700050020B00600200030004020
:103E0C00002C0140C0D8A70004000020001BB70004
:103E1C002507002057EAE068A08601001F85EB51BA
:103E2C0010B572B61A4B93F83030FF2B07D0FFF752
:103E3C0073FF184A184B1288DA6262B610BD164C22
:103E4C00164B41F28732E2621B78E363C4E90D330F
:103E5C00032001F071FC3723A362C820FDF722FD7B
:103E6C00052001F069FC2823A362C820FDF71AFD88
:103E7C00062001F061FC1923A362C820FDF712FD96
:103E8C0001F01CFC064A0023A3621380D1E700BF9B
:103E9C000005002004000020002C01402507002014
:103EAC00B006002070B5164C41F28733E36272B64F
:103EBC00144D154B3C224AF6AA262E60A2621B78A2
:103ECC00E363C4E90D33012001F036FC4B20FDF710
:103EDC00E9FC5023A3624B20FDF7E4FC5A23A362B8
:103EEC004B202E60FDF7DEFC01F0E8FB074A084989
:103EFC0012880023A3620B80E26262B670BD00BF21
:103F0C00002C014000300040250700200400002058
:103F1C00B006002010B572B6144C154A154B4AF673
:103F2C00AA2141F28730E06211605022A2621B7814
:103F3C00E363C4E90D33032001F0FEFB6420FDF7BD
:103F4C00B1FC4623A3626420FDF7ACFC2823A362DA
:103F5C006420FDF7A7FC01F0B1FB074A0749128862
:103F6C000023A3620B80E26262B610BD002C0140FC
:103F7C00003000402507002004000020B00600207F
:103F8C0010B5124C124B41F287313222E162A2621F
:103F9C001B78E363C4E90D33022001F0CDFB9620BE
:103FAC00FDF780FC0B4A4AF6AA211E2311609620CD
:103FBC00A362FDF777FC01F081FB074A07491288E1
:103FCC000023A3620B80E26210BD00BF002C0140F5
:103FDC00250700200030004004000020B00600201F
:103FEC0010B5124C124B41F287312822E162A262C9
:103FFC001B78E363C4E90D33022001F09DFB96208E
:10400C00FDF750FC0B4A4AF6AA215023116096206A
:10401C00A362FDF747FC01F051FB074A07491288E0
:10402C000023A3620B80E26210BD00BF002C014094
:10403C00250700200030004004000020B0060020BE
:10404C002DE9F041154D41F28733EB6272B6144BFA
:10405C00DFF850801B78144FEB63C5E90D337724E0
:10406C004AF6AA26A7FB04300009C8F8006001F044
:10407C0063FB63100A33AB620A20023CFDF712FCAF
:10408C00631CEFD101F01AFB084A0949128800237E
:10409C00AB620B80EA6262B6BDE8F081002C014095
:1040AC002507002000300040CDCCCCCC04000020F3
:1040BC00B0060020002103E00B4B5B584350043149
:1040CC000A480B4B42189A42F6D30A4A02E00023E4
:1040DC0042F8043B084B9A42F9D301F0D1FD01F0B0
:1040EC00D3FFFEF75FFF704754610008000000200B
:1040FC00C8030020C803002054080020FEE700007D
:10410C00836861F300038360704700BF4FF08073D6
:10411C000360704743680A7862F30823436083683E
:10412C004A7862F34103836083688A7862F3CB2315
:10413C008360CB78C26A013B63F31752C26270474B
:10414C00836861F308238360704700BF836843F082
:10415C0008038360704700BF8068C0F3C0007047DD
:10416C00836843F004038360704700BF8068C0F32A
:10417C008000704710B4112917D8DFE811F0120035
:10418C0079007E00830088008D00920097009C00CF
:10419C00A100A600AB00B000B500BA00BF00C4007F
:1041AC007400046963F302040461013A0F2A0DD808
:1041BC00DFE802F00E13181D22272C31363B404548
:1041CC004A4F5408C36A61F3D333C36210BC7047BF
:1041DC00436B61F304034363F8E7436B61F34913E7
:1041EC004363F3E7436B61F38E234363EEE7436B67
:1041FC0061F3D3334363E9E7436B61F318534363D0
:10420C00E4E7436B61F35D634363DFE7036B61F3E7
:10421C0004030363DAE7036B61F349130363D5E724
:10422C00036B61F38E230363D0E7036B61F3D3332A
:10423C000363CBE7036B61F318530363C6E7036BAC
:10424C0061F35D630363C1E7C36A61F30403C36293
:10425C00BCE7C36A61F34913C362B7E7C36A61F38E
:10426C008E23C362B2E7C46863F35754C4609CE7FF
:10427C00046963F3C504046197E7046963F3881464
:10428C00046192E7046963F34B2404618DE70469CC
:10429C0063F30E34046188E7046963F3D134046179
:1042AC0083E7046963F3944404617EE7046963F370
:1042BC005754046179E7046963F31A64046174E781
:1042CC00046963F3DD6404616FE7C46863F302049B
:1042DC00C4606AE7C46863F3C504C46065E7C46876
:1042EC0063F38814C46060E7C46863F34B24C46050
:1042FC005BE7C46863F30E34C46056E7C46863F3C9
:10430C00D134C46051E7C46863F39444C4604CE78F
:10431C00836807298CBF43F000736FF35963836084
:10432C00836861F353438360836862F3145383603F
:10433C00704700BF024B9A6860F3D7529A6070477F
:10434C0000240140836861F396538360704700BF7B
:10435C0020B9034BDA6961F30002DA61704700BFE0
:10436C000000014010B412490B6843F001030B60CC
:10437C000B689B07FCD54B680D4A6FF301034B6030
:10438C00536813F00C0FC3F38101F9D1136823F0B8
:10439C00867323F48033136041F610744FF480104D
:1043AC004FF41F035160D462106310BC93607047CC
:1043BC0000100240030C03F1804303F5043300F0BA
:1043CC001F001A68012303FA00F030EA02030CBF45
:1043DC0001200020704700BF030C03F1804303F55C
:1043EC00043301291A6800F01F0006D0012101FADC
:1043FC0000F022EA00001860704701FA00F0104348
:10440C0018607047030C03F1804303F50433012952
:10441C001A6800F01F0006D0012101FA00F022EA10
:10442C0000001860704701FA00F0104318607047E4
:10443C00042809D8DFE800F0090F151B03000F4B07
:10444C005A6A61F300025A6270470C4B1A6861F3A6
:10445C0000021A607047094B1A6861F310421A6027
:10446C007047064B1A6861F318621A607047034B69
:10447C001A6A61F300021A62704700BF0010024012
:10448C00024B5A6860F307125A60704700100240E2
:10449C00024B5A6860F30A225A60704700100240BF
:1044AC00024B5A6860F3CD225A60704700100240EC
:1044BC00054B5A6860F38F325A605A68C0F380001B
:1044CC0060F31C725A60704700100240134BA0B985
:1044DC005A6860F3104284465A60104B5A6861F374
:1044EC0095425A605A68C1F3011060F35E725A60CB
:1044FC00DA6A6CF31A62DA6270475A6842F48032F4
:10450C005A605A6801280BBF6FF3514242F40032D3
:10451C004FF0020C4FF0000C5A60DEE70010024026
:10452C00024B5A6860F301025A6070470010024057
:10453C00024B5868C0F38100704700BF0010024066
:10454C0038B53F4D6B6813F00C0F0446C3F3810272
:10455C0028D0022A2FD03B4B236039483A4A416875
:10456C003A4DC1F30311515CCB4063604168C1F318
:10457C0002211144097C23FA01F1E1604168C1F385
:10458C00C221695CCB40A36045684168C5F30070EB
:10459C00C1F3813141EA80010A44127EB3FBF2F38C
:1045AC00236138BD6B6D9805D5D52B6B9901D2D590
:1045BC00274B2360D1E76968EB6A002BC1F30041FC
:1045CC001DDAEA6AEB6AC2F3031CEA6AC3F3082336
:1045DC0002F0070269B369681E4811F4003F1949DB
:1045EC0008BF08460021A3FB000503FB01F10CFAF0
:1045FC0002F20023FCF764FD03462060ADE76B6814
:10460C006A6812F0C04FC3F38343C2F341700CD1FC
:10461C000F2B0AD0023319B1094A526892030AD5FA
:10462C000C4800FB03F3236097E7013303EB001303
:10463C00F1E70848D7E7034800FB03F323608CE756
:10464C000010024000127A00146100082461000876
:10465C00006CDC0200093D00012805D0054B5A6DA9
:10466C006FF305125A657047024A536D43F03003DD
:10467C00536570470010024010B404680C490022C6
:10468C00C3B26FF300040460083B026042608260B6
:10469C00C260A2F13332A2FB03231B09486810BC91
:1046AC009B000F2202FA03F303434B60704700BFD9
:1046BC0000000240036861F300030360704700BF11
:1046CC00034B1B68034214BF01200020704700BF3E
:1046DC00000002400023C0E90033C0E9023303822A
:1046EC00704700BF03684BF6EF721340036002681B
:1046FC000B891343036003684A7C62F30D33036038
:10470C000368CA7B62F38B23036003688A7B62F3C2
:10471C000923036003684A7B62F3C71303600368D1
:10472C000A7B62F3861303600A7C036862F3451309
:10473C000360D1E9002310B44C894460826010BC42
:10474C00C3607047014BD860704700BF0020024027
:10475C00024B0349034A59605A60704700200240DB
:10476C0023016745AB89EFCD024A136943F08003FF
:10477C0013617047002002401B4A136943F0020387
:10478C0013615061136943F040031361D368D90777
:10479C0004D4D3685B0720D5012011E04FF080438F
:1047AC00D168C80712D4D168490713D4D268D2068D
:1047BC0003F1FF334CBF02200320002B08BF042061
:1047CC00094B1A696FF341021A617047013BE7D13B
:1047DC000420F5E7013B0120EFE7D36813F0100F3D
:1047EC0014BF02200320EBE700200240194A136992
:1047FC0043F0010313610160D368D90704D4D36873
:10480C005B0720D5012011E04FF48013D168C80755
:10481C0012D4D168490713D4D268D20603F1FF33FE
:10482C004CBF02200320002B08BF0420094B1A693F
:10483C006FF300021A617047013BE7D10420F5E7E2
:10484C00013B0120EFE7D36813F0100F14BF0220D7
:10485C000320EBE7002002400B88002B43D02DE90E
:10486C00F0434FF0000E032601251FFA8EFC4FEA91
:10487C004C0213F0010F06FA02F705FA0CF80EF1D0
:10488C00010E2CD0046824EA070404608C79D0F85B
:10489C000090944044EA09040460446824EA080443
:1048AC0044600C79D0F8048004FA0CFC4CEA08043F
:1048BC004460846824EA07048460CC79D0F808C08A
:1048CC00944044EA0C048460C46824EA0707C76077
:1048DC0091F805C0C4680CFA02F22243C2605B086E
:1048EC00C3D1BDE8F083704701F007039B00C908F2
:1048FC0002FA03F20BD0416A4FF00F0C0CFA03F3DF
:10490C0021EA03034362436A1A4342627047016A15
:10491C004FF00F0C0CFA03F321EA03030362036A52
:10492C001A430262704700BF1F4BDB68C3F30223BC
:10493C0000B5C3F1070EBEF1040F03F1040C28BF40
:10494C004FF0040EBCF1060F21D9033B4FF0FF3C96
:10495C000CFA03FC22EA0C024FF0FF3C0CFA0EFCA2
:10496C0021EA0C019940002841EA020112DB0F4AAE
:10497C0009011318C9B283F800130123410900F08F
:10498C001F0003FA00F042F821005DF804FB00223E
:10499C001346E1E7064B00F00F0009010344C9B2CE
:1049AC0019765DF804FB00BF00ED00E000E100E0CB
:1049BC00FCEC00E008B52E4B98421CD02D4B9842D5
:1049CC0023D02D4B98422AD02C4B984209D02C4BFB
:1049DC0098422ED02B4B984235D02B4B98423CD042
:1049EC0008BD2A480121FFF70DFDBDE80840274806
:1049FC000021FFF707BD26480121FFF703FDBDE8A5
:104A0C00084023480021FFF7FDBC22480121FFF795
:104A1C00F9FCBDE808401F480021FFF7F3BC1E4815
:104A2C000121FFF7EFFCBDE808401B480021FFF710
:104A3C00E9BC1A480121FFF7E5FCBDE8084017481E
:104A4C000021FFF7DFBC16480121FFF7DBFCBDE8B6
:104A5C00084013480021FFF7D5BC12480121FFF78D
:104A6C00D1FCBDE808400F480021FFF7CBBC00BFCC
:104A7C00002C0140000400400010004000200040C9
:104A8C000040014000440140004801400800100073
:104A9C000B000C00010010000400100010000C00B2
:104AAC0011000C0012000C00036861F3C7130360C3
:104ABC00704700BF062909D8DFE801F013080E087B
:104ACC0009080400C36962F3CB23C3617047C3694F
:104ADC0062F3C303C3617047836962F3CB238361C1
:104AEC007047836962F3C30383617047062909D851
:104AFC00DFE801F0090E13181D220400036A62F3AB
:104B0C000C3303627047036A62F30003036270475D
:104B1C00036A62F3820303627047036A62F304134D
:104B2C0003627047036A62F3861303627047036A79
:104B3C0062F3082303627047036A62F38A230362F9
:104B4C00704700BF2DE9F04186B0054601A8174615
:104B5C001E468846FFF7F4FCDDE90334114A954202
:104B6C0008BF1C4604EB84046400B4FBF8F10E4C43
:104B7C00A4FB0134E40804EB8403A1EB43010429F6
:104B8C00AB6888BF0134A4B264F30F03AB60EB686D
:104B9C0067F30C33EB602B6966F30D332B6106B0B6
:104BAC00BDE8F08100380140CDCCCCCCC36861F3BA
:104BBC004D33C360704700BFC36861F3C303C36068
:104BCC00704700BFC36861F38203C360704700BFC6
:104BDC00436961F3C7134361704700BF436961F3D5
:104BEC00C3034361704700BF064B0748B3F806C0C8
:104BFC000649074AA0F800C018885B880880138013
:104C0C00704700BF28070020C8060020CC060020F3
:104C1C003806002030B5082387B0002203214FF05E
:104C2C009040FCF7BBFE4023002203214FF0904044
:104C3C00FCF7B4FE01214FF4A010FFF7CDFB334875
:104C4C00334CFFF719FD01A8FFF744FD314B324AF5
:104C5C002E48019301A940F201234FF480250492C0
:104C6C00ADF81430CDE90245FFF73CFD2748012192
:104C7C00FFF720FD01212948FFF7AEFB0720FFF7C6
:104C8C0017FC6846FFF742FA254B26480093694605
:104C9C00FFF740FA2348032301220621FFF76AFAA3
:104CAC00032319461F480222FFF764FA03231A460E
:104CBC001C481121FFF75EFA072304221021194822
:104CCC00FFF758FA0120FFF735FB012215480721A1
:104CDC00FFF71EFB13480121FFF732FA114801219F
:104CEC00FFF70EFA0F48FFF731FA0E48FFF734FAC8
:104CFC000028FAD10B480B4CFFF732FA2046FFF78D
:104D0C0035FA0028FAD107B030BD00BF08000240C8
:104D1C00280700204C240140000101010900180063
:104D2C00010100040024014048F2E80303FB00F0F9
:104D3C000028B8BF00F6FF70054B0013C0F54850B3
:104D4C0083FB0023C017A0EBE300193000B27047BF
:104D5C00310CC33038B5164D164C6B6C6B64204659
:104D6C00FFF728FE144B41210B22A16122621A7815
:104D7C00A2624FF6FF73E3626269104B002142F0AE
:104D8C000102626103F8041B0D4A6162EA640D4A78
:104D9C002B651378AB64E36843F40073E36023681A
:104DAC0043F0010340F68B1223606A6438BD00BFE8
:104DBC000000024000040040C20300203007002025
:104DCC0034040040BE03002038B51D4D1D4C6B6CE7
:104DDC0043F010036B642046FFF7ECFD60210323C6
:104DEC00194AA16123621278184BA2624C2101224C
:104DFC00E1621A7063691649164A43F00103636154
:104E0C00154BE9642A655B781733AB646B6C43F024
:104E1C0002036B646B6C43F008036B646B6C43F0C4
:104E2C0001036B64E36843F40073E360636C43F465
:104E3C0000436364236843F00103236038BD00BF63
:104E4C00000002400004004018070020300700203A
:104E5C003404004034040020C2030020024B1869C3
:104E6C0000F01000704700BF0004004802481023F7
:104E7C0001220221FCF79EBD00040048FEE700BFA2
:104E8C00FEE700BFFEE700BFFEE700BF704700BFB4
:104E9C00704700BF704700BF704700BF10B50220BD
:104EAC00FFF70EFC012800D010BD054C6060FFF729
:104EBC009BFE0820FFF704FC012808BF606010BDB2
:104ECC000000024008B5264B1B78002B39D14FF45B
:104EDC008040FFF7F5FB012811D04FF40050FFF78D
:104EEC00EFFB01281ED04FF40040FFF7E9FB01282F
:104EFC0000D008BD1B4B4FF480525A6008BD1A4BB2
:104F0C001B78002BE9D0194A1649136A4FF48040DC
:104F1C0043F00203136248604FF40050FFF7D0FBDC
:104F2C000128E0D10F4B4FF480525A605A6C6FF34A
:104F3C0000025A64FEF724FE0D4B4FF400421A6136
:104F4C00D1E7084B4FF480525A605A6C6FF3000251
:104F5C005A64FEF715FE064B4FF400421A6108BD69
:104F6C00C205002000000240C305002000040040E0
:104F7C000004014008B50D4A0D4B12685B6AB3EB97
:104F8C00520F07D90B4B4FF400125A61BDE8084081
:104F9C00FCF79ABF00F052F8074B1B78834200D005
:104FAC0008BD044B4FF400125A6108BD40060020A6
:104FBC00001000400004014052000020024B4FF64C
:104FCC00FE721A61FDF754BD00200040024B002216
:104FDC001A61FCF739BF00BF00440140034B4FF688
:104FEC00FE714FF6FD7219611A6170470040014065
:104FFC00704700BF074B1A69910744BF4FF6FD720B
:10500C001A61044B1A69D20744BF4FF6FE721A613B
:10501C00704700BF00040040064A0749136801337B
:10502C0013604B691B0400D470474FF400434B6171
:10503C00FDF704BC3408002000040140024BD86981
:10504C00C0F38070704700BF00000140044B1A6829
:10505C004FF4001122F400121A605961704700BF1E
:10506C0000040140024A136843F4001313607047B4
:10507C00000401400F4B1B68B3F5C87F10D20E4AD9
:10508C00D36923F00403D3610C4B0D4A1B78002B1E
:10509C000CBF4FF4001100215B059160D360704789
:1050AC00B3F5167FF0D9044AD36943F00403D361F6
:1050BC00EAE700BF4006002000000140520000203B
:1050CC00000401402DE9F0430029B4BFCE1C0E466C
:1050DC0026F00303073383B023F0070300AFADEBD7
:1050EC00030DB6106D4688468146144600213246A3
:1050FC00284600F0EDFFB8F1030F17DD4846291FD5
:10510C000022837890F8038090F800E090F801C0BA
:10511C001B0443EA086343EA0E03013243EA0C23FF
:10512C00964241F8043F00F10400EADC3E60FFF7D0
:10513C000FFBC4F30903EBB100237B607B683A6877
:10514C009A4211D978687B6804EB800055F82310DB
:10515C00FFF74CFB0320FFF7F5FA7B6801337B600C
:10516C007A683B689A42EDD3FFF7FEFA0C37BD46DE
:10517C00BDE8F0832046FFF7FFFADDE7002A30DDBB
:10518C00531E072B10B501F1010421D9031B022B6F
:10519C001ED922F0030E8E440B46441AD3F800C0DD
:1051AC0044F803C004337345F8D1940722F0030389
:1051BC000DD0CC5CC4545C1CA24208DD023311F847
:1051CC0004C000F804C09A4201DDCA5CC25410BD90
:1051DC00431E1A44201AC15C03F8011F9342FAD1F2
:1051EC0010BD704762B670471C4B40F2531210B59D
:1051FC001A60FFF7B7F801210020FFF719F9012019
:10520C00FFF7D8F801280446F9D100201D21FFF73B
:10521C005DF921460220FFF70BF91920FFF7CAF8B8
:10522C0001280446F9D10020FFF72AF90020FFF7E6
:10523C0037F90020FFF72CF92046FFF70DFA022072
:10524C00FFF76EF9FFF774F90228FBD10020FFF786
:10525C0003FABDE8104000F043BD00BF002002403F
:10526C00084B10B44CF6CC4245F255541C6003204C
:10527C001A604FF47A614AF6AA22586010BC996001
:10528C001A6070470030004038B53F483F4C012150
:10529C00FFF7A2F80025682341F2873146F6680231
:1052AC00E1622046A5622946A261E3610122FFF773
:1052BC0001FC204601220221FFF7FCFB01222046C3
:1052CC000421FFF7F7FB20460121FFF7EDFB636C90
:1052DC002F483C2262F3070363640121FFF77CF83B
:1052EC002C4C2D480121FFF777F8022319462A464A
:1052FC002046FCF753FB2A46204601230221FCF7EB
:10530C004DFB80232A4602214FF09040FCF746FBD0
:10531C00204602220121FFF7E7FA29462046022205
:10532C00FFF7E2FA022207214FF09040FFF7DCFA78
:10533C002A464FF4806302214FF09040FCF72EFB7D
:10534C002A464FF4007302214FF09040FCF726FBE5
:10535C004FF480732A4602214FF09040FCF71EFB5D
:10536C0002220A214FF09040FFF7BEFA02220921D7
:10537C004FF09040FFF7B8FABDE838400222082100
:10538C004FF09040FFF7B0BA0B001800002C014012
:10539C001100140000040048120014002DE9F0471D
:1053AC004D4CFFF721FF102501214FF4A010FFF702
:1053BC0013F884F80B534FF40068C4F80080FFF71F
:1053CC0063FF46480121FFF707F8454B45484FF668
:1053DC00FF774FF03B09DF620121C3F82890FEF7FD
:1053EC00FBFF414B32224FF0770ADA62C3F828A058
:1053FC00302384F813334FF4002323603B480121FE
:10540C00FEF7EAFF01214FF4C010FEF7E5FF00267E
:10541C000223002203214FF09040FCF7BFFA202317
:10542C00324603214FF09040FCF7B8FA84F80C6335
:10543C004FF48053236001213046FEF789FF2C483E
:10544C000121FEF7C9FF2B4B2B48DF62C3F828A0C4
:10545C001A6842F080021A600121FEF7BDFF274B4B
:10546C004FF4FA72DA62C3F8289084F815634FF49B
:10547C0000132360DFF8889022480121FEF7ACFF6F
:10548C0021480121FEF7A8FF2B463246484602214F
:10549C00FCF784FA484601220421FFF725FA012182
:1054AC004FF4A010FEF798FF184B40F68A125A647E
:1054BC0084F80B53C4F80080A3F5FE33DF629D62C1
:1054CC001A6842F080021A601A6842F001021A60EF
:1054DC00BDE8F04700F06ABB00E100E004001C00EE
:1054EC000010004008001C000020004011001400B7
:1054FC00120018000048014011001800004401403F
:10550C00000400481200140001001C0000000240BE
:10551C00014B5863704700BF002C0140014B98634E
:10552C00704700BF002C0140014BD863704700BF8F
:10553C00002C0140024A536943F001035361704748
:10554C00002C0140024B0022DA625A62704700BF05
:10555C000004004010B5384C012220460021FFF712
:10556C00C5FA204601220221FFF7C0FA204601228B
:10557C000421FFF7BBFA012211462046FFF7B6FAC9
:10558C00204601220321FFF7B1FA20460122052112
:10559C00FFF7ACFA2268294B294842F0010222603D
:1055AC00626C42F400426264626942F00102626120
:1055BC001968244A41F001011960596941F001014F
:1055CC005961D96821F00101D960016841F00101EC
:1055DC000160116841F0010111605169A3F592332A
:1055EC0041F0010151611A6842F001021A605A69D6
:1055FC0042F001025A61DA6842F00102A4F59434D7
:10560C00DA60FFF707FB012200212046FFF76EFA54
:10561C0023680D4A43F001032021236082F807130D
:10562C008023136002F1C04202F50C52136843F45C
:10563C000043136010BD00BF002C0140004401402A
:10564C00004801400010004000E100E070B54FF050
:10565C00904420464FF4806300220121FCF79EF910
:10566C004FF48060A0624FF40073204600220121A9
:10567C00FCF794F94FF400700F4DA0624FF4807357
:10568C00204600220121FCF789F902234FF4807097
:10569C001946A06200222846FCF780F9284601230F
:1056AC0000220221FCF77AF920468023BDE87040E5
:1056BC0000220221FCF772B90004004870B51D4E9F
:1056CC0002230022012130464FF09044FCF766F98A
:1056DC0002204FF4806300220121B0622046FCF7C7
:1056EC005DF901234FF480601D4619460022A0622B
:1056FC003046FCF753F94FF400730022294620463C
:10570C00B562FCF74BF94FF4007180230022A162C3
:10571C0020462946FCF742F98023A36200224FF46D
:10572C00807329462046FCF739F94FF48073A36245
:10573C0070BD00BF000400480138F8B5052845D8F5
:10574C00DFE810F045008400F900C3002E010600CC
:10575C00BF4E01231D464FF090441946002230469F
:10576C00FCF71CF94FF40073002229462046B56261
:10577C00FCF714F94FF400728023A2622946002230
:10578C002046FCF70BF98023A36100224FF48073B1
:10579C0029462046FCF702F9AE4A127D4FF480737D
:1057AC00A3620223002A40F02F8129463046FCF7E1
:1057BC00F5F80223B3624FF48063002202214FF00C
:1057CC009040FCF7EBF8A44BA44ADA61F8BD4FF01B
:1057DC0090448023002201212046FCF7DFF8802032
:1057EC009B4DA0624FF48073002201212046FCF7F0
:1057FC00D5F801234FF4807019460022A0620126CF
:10580C002846FCF7CBF84FF400730022AE6131460A
:10581C002046FCF7C3F88F4A127D4FF40073A36245
:10582C000223002A40F0FC8031462846FCF7B6F8EB
:10583C000223AB624FF48063002202214FF09040B0
:10584C00FCF7ACF8844B864ADA61F8BD804D4FF01A
:10585C00904402230022012128460227FCF79EF8DF
:10586C004FF48063002201212046AF62FCF796F8CA
:10587C0001234FF480621946A262284600220126B9
:10588C00FCF78CF84FF400730022AE6131462046D1
:10589C00FCF784F86F4A127D4FF40073A3628023E7
:1058AC00002A40F0C98031462046FCF777F8802367
:1058BC00A3624FF48073002202214FF09040FCF75A
:1058CC006DF8654B674ADA61F8BD4FF09044802360
:1058DC00002201212046FCF761F880205C4DA0627B
:1058EC004FF48073002201212046FCF757F84FF447
:1058FC00807102230022A162284601210226FCF7B6
:10590C004DF84FF480630022AE6101212046FCF774
:10591C0045F8504A127D4FF48063A3620123002A9C
:10592C0040F0848019462846FCF738F80123AB6216
:10593C004FF4007380E7464E01231D464FF0904410
:10594C00194600223046FCF729F84FF40073002268
:10595C0029462046B562FCF721F84FF40072022369
:10596C00A2622946002230460227FCF717F84FF4B2
:10597C0080630022B76129462046FCF70FF8354AB0
:10598C00127D4FF48063A3628023002A5AD12946EA
:10599C002046FCF703F88023A3624FF480730CE7D6
:1059AC002B4D4FF090440223002201212846022661
:1059BC00FBF7F4FF4FF48063002201212046AE6216
:1059CC00FBF7ECFF4FF480628023A26201210022DE
:1059DC002046FBF7E3FF8023A36100224FF4807382
:1059EC0001212046FBF7DAFF1A4A127D4FF480732F
:1059FC00A362012372B919462846FBF7CFFF012396
:105A0C00AB624FF4007356E7002219463046FBF7A1
:105A1C00C5FFD0E6002231462846FBF7BFFFF0E772
:105A2C00002219462846FBF7B9FF03E7002231464E
:105A3C002846FBF7B3FF7BE7002239462046FBF7ED
:105A4C00ADFF36E7002239462046FBF7A7FFA4E757
:105A5C00000400480005002000000140C500004083
:105A6C00D5000040E500004070B51D4E0223002219
:105A7C00012130464FF09044FBF790FF02204FF489
:105A8C00806300220121B0612046FBF787FF0123D0
:105A9C004FF480601D4619460022A0623046FBF789
:105AAC007DFF4FF40073002229462046B561FBF7B9
:105ABC0075FF4FF4007180230022A1622046294615
:105ACC00FBF76CFF8023A36100224FF480732946FF
:105ADC002046FBF763FF4FF48073A36270BD00BFD9
:105AEC000004004870B5284C227DBABB274D022318
:105AFC0001212846FBF752FF0223AB6200224FF430
:105B0C00806302214FF09040FBF748FF227D9ABB47
:105B1C001E4D012319462846FBF740FF0123AB62BB
:105B2C004FF40073002202214FF09040FBF736FF38
:105B3C00227D8023CAB901214FF09040FBF72EFF44
:105B4C004FF0904380229A62BDE870404FF480730E
:105B5C00002202214FF09040FBF720BF02230B489C
:105B6C0000221946FBF71AFFC8E7002202214FF06A
:105B7C009040FBF713FFE7E70448012300220221C2
:105B8C00FBF70CFFCCE700BF000500200004004829
:105B9C00054BDA696FF30002DA611862DA6942F0D8
:105BAC000102DA61704700BF0000024030B52B489B
:105BBC002B4D2C4C89B00121FEF70EFC2A480121FB
:105BCC00FEF70AFC01214FF4A010FEF705FC274B51
:105BDC0001A928464022CDE90123FEF73DFE002213
:105BEC0006212846FEF780FE2046FEF745FD03A859
:105BFC00FEF770FD1E4A1F4B2046CDE903321E4CAA
:105C0C001E4A002503A94FF48073CDE90523ADF896
:105C1C001C50FEF767FD2B462A4620464FF4E13117
:105C2C00FEF790FF20460121FEF7C6FF204601211A
:105C3C00FEF7C8FF20460121FEF7D0FF20460121C8
:105C4C00FEF7C6FF20460121FEF7B0FF2A460321CE
:105C5C000A20FEF769FE09B030BD00BF0E00180027
:105C6C00000400481C000240120014000001020154
:105C7C00CC040020043801400038014010003100F1
:105C8C0030B414490B6843F001030B600B689B079D
:105C9C00FCD54B680F4A6FF301034B60536813F04C
:105CAC000C0FC3F38101F9D113680B480B4C23F093
:105CBC00867323F48033136041F610754FF4801310
:105CCC005160D56213634FF41F039360846030BC42
:105CDC00704700BF0010024000ED00E0001000080B
:105CEC0010B5FEF725FC60B1022816D02C482D4BC0
:105CFC002D495B682D4AC3F30313CB5CD84010606D
:105D0C0010BD284B5A6D9205F0D51A6B244B2848C0
:105D1C0012F0007F08BF1846E9E7224B5968DA6A8F
:105D2C00002AC1F300411CDAD86ADC6ADA6AC0F3D3
:105D3C00031EC4F3082402F0070259B35B681D4824
:105D4C0013F4003F164B4FF0000108BF18460EFA33
:105D5C0002F20023A4FB000E04FB01F1FBF7B0F9E7
:105D6C00C5E758685B6813F0C04FC0F38340C3F3BA
:105D7C0041720BD10F2809D0023019B1094B5B6865
:105D8C009B0309D50B4B03FB00F0B0E7013000EB94
:105D9C000210F2E70748DAE7014B03FB00F0A6E735
:105DAC0000127A000010024034610008C403002085
:105DBC00006CDC0200093D002DE9F047089E0D4601
:105DCC0004468846002B4DD18A42944668D9B2FAD3
:105DDC0082F252B101FA02F3C2F1200120FA01F170
:105DEC000CFA02FC41EA030894404FEA1C45210CD2
:105DFC00B8FBF5FE1FFA8CF705FB1E8341EA034343
:105E0C000EFB07F199420BD91CEB03030EF1FF308B
:105E1C0080F01E81994240F21B81AEF1020E634468
:105E2C005B1AA4B2B3FBF5F005FB103344EA034450
:105E3C0000FB07F7A7420AD91CEB040400F1FF335F
:105E4C0080F00881A74240F2058164440238E41BCB
:105E5C0040EA0E4000211EB1D4400023C6E90043A5
:105E6C00BDE8F0878B4208D9002E00F0EE800021AF
:105E7C00C6E900050846BDE8F087B3FA83F10029AE
:105E8C004AD1AB4202D3824200F2F980841A65EB0C
:105E9C00030301209846002EE2D0C6E90048DFE754
:105EAC0002B9FFDEB2FA82F2002A40F09180A1EB37
:105EBC000C054FEA1C471FFA8CFE0121B5FBF7F3CA
:105ECC0007FB1350250C45EA00450EFB03F0A842D6
:105EDC0008D91CEB050503F1FF3802D2A84200F2E9
:105EEC00CB8043462D1AA4B2B5FBF7F007FB105537
:105EFC0044EA05440EFB00FEA64508D91CEB04043D
:105F0C0000F1FF3502D2A64500F2BB802846A4EB77
:105F1C000E0440EA03409EE7C1F120078B4022FAB1
:105F2C0007FC4CEA030C20FA07F405FA01F31C43B6
:105F3C00FD404FEA1C4900FA01F3B5FBF9F8200CBF
:105F4C001FFA8CFE09FB185540EA054508FB0EF0BC
:105F5C00A84202FA01F20BD91CEB050508F1FF3A35
:105F6C0080F08880A84240F28580A8F10208654440
:105F7C002D1AA4B2B5FBF9F009FB105544EA0545FE
:105F8C0000FB0EFEAE4508D91CEB050500F1FF34F5
:105F9C006CD2AE456AD90238654440EA0840A0FB91
:105FAC000294A5EB0E05A542C846A64656D353D07F
:105FBC005EB1B3EB080265EB0E0505FA07F722FAA2
:105FCC0001F3CD401F43C6E900750021BDE8F08701
:105FDC00C2F1200320FA03F10CFA02FC25FA03F3B8
:105FEC0095400D434FEA1C471FFA8CFEB3FBF7F1AB
:105FFC0007FB11302B0C43EA004301FB0EF09842D7
:10600C0004FA02F408D91CEB030301F1FF382FD278
:10601C0098422DD9023963441B1AADB2B3FBF7F089
:10602C0007FB103345EA034500FB0EF3AB4208D9DE
:10603C001CEB050500F1FF3816D2AB4214D902381F
:10604C006544ED1A40EA014138E73146304607E72E
:10605C008646E5E61846FAE64B45A9D2B9EB0208A6
:10606C0064EB0C0E0138A3E74046EAE7204694E7C0
:10607C004146D1E7D0467BE7023B654432E7084610
:10608C0009E76444023842E770B50D4D0D4C641BB2
:10609C00A4100026A64209D10B4D0C4C00F020F8A0
:1060AC00641BA4100026A64205D170BD55F8043B14
:1060BC0098470136EEE755F8043B98470136F2E76E
:1060CC004C6100084C6100084C61000850610008EC
:1060DC0002440346934200D1704703F8011BF9E7D1
:1060EC00F8B500BFF8BC08BC9E467047F8B500BFB9
:0860FC00F8BC08BC9E46704789
:10610400191B12131D1516171A090A0B1E0D0E0F53
:106114000000000000000000010203040607080953
:10612400000000000102030402040608020C081027
:106134000000000000000000010203040607080933
:0861440080FCFF7F0100000058
:04614C002511000811
:046150000111000831
:10615400007C0008871387133C007800C800D00730
:106164004C046C07DC0564004A013C00900100000B
:10617400000000009001000000000000E80300009F
:10618400000000000000000000000000000000000B
:10619400204E0000A08601000206100114004600F3
:1061A400DC05010501010100D430000005010A00ED
:1061B400E803000010270000000000000A000000AF
:1061C4000000000064000000000000000000000067
:1061D40000000000000000001027000050C3000071
:1061E400B400D007D0070000B400B700BA00BD0067
:1061F400C100C400C700CA00CD00D000D300D6003F
:10620400D900DC00E000E300E600E900EC00EF0068
:10621400F200F500F700FA00FD0000010301060199
:1062240009010B010E0111011301160119011B01D2
:106234001E0120012301250128012A012C012F011F
:1062440031013301350138013A013C013E0140017D
:10625400420144014601470149014B014D014E01F0
:1062640050015101530154015601570158015A017B
:106274005B015C015D015E015F016001610162011E
:1062840063016301640165016501660166016701DB
:1062940067016701680168016801680168016801B4
:1062A40068016801680167016701670166016601A9
:1062B40065016501640163016301620161016001BB
:1062C4005F015E015D015C015B015A0158015701E8
:1062D400560154015301510150014E014D014B012E
:1062E4004901470146014401420140013E013C018C
:1062F4003A0138013501330131012F012C012A0102
:1063040028012501230120011E011B011901160189
:10631400130111010E010B01090106010301000122
:10632400FD00FA00F700F500F200EF00EC00E900D0
:10633400E600E300E000DC00D900D600D300D00082
:10634400CD00CA00C700C400C100BD00BA00B70038
:10635400B400B100AE00AB00A700A400A1009E00F1
:106364009B009800950092008F008C0088008500A7
:1063740082007F007C0079007600730071006E005B
:106384006B006800650062005F005D005A00570002
:10639400550052004F004D004A004800450043009C
:1063A40040003E003C003900370035003300300027
:1063B4002E002C002A0028002600240022002100A0
:1063C4001F001D001B001A00180017001500140000
:1063D4001200110010000E000D000C000B000A004A
:1063E400090008000700060005000500040003007A
:1063F400030002000200010001000100000000008F
:106404000000000000000000000000000000010087
:106414000100010002000200030003000400050063
:10642400050006000700080009000A000B000C0024
:106434000D000E00100011001200140015001700CA
:1064440018001A001B001D001F0021002200240058
:10645400260028002A002C002E00300033003500CE
:10646400370039003C003E0040004300450048002E
:106474004A004D004F005200550057005A005D007D
:106484005F006200650068006B006E0071007300BD
:10649400760079007C007F008200850088008C00F3
:1064A4008F009200950098009B009E00A100A4001C
:1064B400A700AB00AE00B1003C001E03030064194A
:1064C4000000000001000000000000003200000095
:1064D40000000000000000000000000000000000B8
:1064E4001027000050C3000002003C006E00D007DB
:1064F40064000500E8030614013278004B00010033
:106504005A005A001E000201FA000000204E20002A
:0865140050C3110700127A00C8
:107BE000415433324445565F463432310000000080
:107BF0000000000000000000000000000000000085
:04000005080040C1EE
:00000001FF
